:1000000012C02CC02BC07FC029C028C027C026C06A
:1000100025C025C023C022C021C020C01FC01EC0D3
:100020001DC01CC01BC011241FBECFE5D4E0DEBF25
:10003000CDBF10E0A0E6B0E0E2EDF3E002C0059035
:100040000D92A036B107D9F710E0A0E6B0E001C0EC
:100050001D92A83EB107E1F706D1B9C1D1CF1F92D9
:100060000F920FB60F9211242F933F934F935F93EC
:100070008F939F932091E3003091E4004091E5003D
:100080005091E6002F5F3F4F4F4F5F4F9091E70039
:10009000892F8D5F8093E7008D3738F09A579093C2
:1000A000E7002F5F3F4F4F4F5F4F2093E3003093A8
:1000B000E4004093E5005093E6009F918F915F919B
:1000C0004F913F912F910F900FBE0F901F90189559
:1000D00020E030E014C0FC0143E0EE0FFF1F4A9522
:1000E000E1F7E20FF31FEE59FF4F108201968830BF
:1000F000910589F72F5F3F4F2830310519F080E0D7
:1001000090E0E9CF08951F920F920FB60F9211243D
:100110002F933F934F936F937F938F939F93EF937F
:10012000FF93939895984091600020E030E0642F11
:1001300070E0F90183E0EE0FFF1F8A95E1F7E60F0B
:10014000F71FEE59FF4F9081949895BB82B3907C36
:100150008F73982B92BB949A2F5F3F4F28303105B5
:1001600041F788B3887F842B88BB959A4F5F47708F
:1001700040936000939AFF91EF919F918F917F91AF
:100180006F914F913F912F910F900FBE0F901F9045
:10019000189540E050E020E030E05F9BFECF8CB14E
:1001A00090E08F3F910531F45F9BFECF8CB190E0E2
:1001B000009779F3FA0193E0EE0FFF1F9A95E1F7AC
:1001C000E20FF31FED55FF4F80832730310541F4D7
:1001D0004730510511F4F1D0DCCF4F5F5F4FDBCFDB
:1001E0002F5F3F4FDACFEF92FF920F931F93CF9382
:1001F000DF93F82EE22E062F10E0C42FD0E090E01F
:10020000B801AE01C6D0882339F1B80123E0660FEA
:10021000771F2A95E1F7EE2079F0FB01EC0FFD1F27
:10022000EE59FF4F208181E090E002C0880F991FB6
:10023000FA94E2F7282B0FC0FB01EC0FFD1FEE59DB
:10024000FF4F208181E090E002C0880F991FFA944F
:10025000E2F7809528232083DF91CF911F910F91A2
:10026000FF90EF900895DF92EF92FF920F931F930C
:1002700012BE83B7836083BF89B7816089BF8BE07B
:1002800083BD85B5856085BD85B5886085BD14BC99
:1002900089B7806889BF12BA18BA15BA8FEF81BBC7
:1002A00087BB84BB10BC89E189B986E880BD88E141
:1002B0008AB978946EDF20E0EE24E394DD24DA94AA
:1002C00014C080E090E0422F50E0FC0133E0EE0FDC
:1002D000FF1F3A95E1F7E40FF51FEE59FF4FD0826B
:1002E00001968830910589F72F5F283050F3E0920E
:1002F000A2002091E3003091E4004091E50050918C
:10030000E6008091E3009091E400A091E500B091B7
:10031000E600821B930BA40BB50B88589341A040B9
:10032000B04078F31092A200D3DEFF2430C0812FBA
:10033000602F4F2D21E057DFE092A2002091E300D3
:100340003091E4004091E5005091E6008091E30097
:100350009091E400A091E500B091E600821B930B20
:10036000A40BB50B84369105A105B10578F3109265
:10037000A2001F5F1830D9F60F5F083011F010E0AF
:10038000D6CFF39488E0F81611F420E09ACF00E07D
:10039000F6CF089778F477FD0DC06830710554F4F6
:1003A00057FD08C090E0483051050CF091E081E025
:1003B000982701C090E0892F0895A2E6B0E0E3EA13
:1003C000F0E080E401900D928150E1F70895F894F7
:0203D000FFCF5D
:00000001FF
